:1000000012C0189518951895189518951895189563
:100010001895189518951895189518951895189578
:100020001895189518958FE58DBFC0E4E0E44E2E25
:1000300084E08EBFD4E0F4E05F2EEEEFF3E0A0E6C4
:10004000B0E0A89584B7082E877F84BF88E1992700
:1000500081BD91BD88278D933197E9F73CD2662405
:100060008DEF87BB8CEF84BB8FEF81BB80E088BBBB
:10007000C19A80E085BB80E082BBE2E9F0E080E4E9
:1000800072D258E0C895802D68D231965A95D1F732
:1000900004C010181C1E1E1C1810E2EBF0E088E4CF
:1000A00062D258E0C895802D58D231965A95D1F732
:1000B00004C01F1F1F1F1F1F1F1FE2EDF0E080E580
:1000C00052D258E0C895802D48D231965A95D1F732
:1000D00004C020202020201F1F1F83E886B980E451
:1000E00087B98CE040D2DDD1E8EBF9E0D2D1D7D1AD
:1000F000EAECF9E0CED1E8E2F0E0AEE6B0E091E083
:100100003ED400916E000E3C08F00DC0CAD1E8EB61
:10011000F9E0BFD1C4D1ECEDF9E0BBD185B78F7D5B
:10012000806A85BF889584E690E049D280916E0010
:10013000815080936E00E8E2F0E0AEE6B0E091E03E
:100140007BE70CD4E2E0F0E0BDD1ABD1E2E3F0E03C
:10015000A6E7B0E091E013D48091760080936F0021
:1001600081E0809368008FE716E0AAD180E0F5D1A6
:10017000809172008F778093720080916F008093DE
:10018000750022D18FE711E09BD1EEEEF9E081D12D
:100190008FE717E095D12FD181E08093760043D18E
:1001A000ECEAF9E05CD3E9E6F0E05AD224D3EDE0E2
:1001B000F0E022D2A0E7B0E0DC9280917000809362
:1001C000750002D18FEB11E07BD1E4EFF9E061D152
:1001D00012D1B998A2E7B0E09C9196FF04C0B19B00
:1001E0000EC09F7B9C93B1990AC088E29F93992788
:1001F000E6D19F91B19903C090649C939ED00091E9
:100200006800013009F048C0C598A0E6B0E0ECEF06
:10021000F9E0E4D18FEB1EE053D1A0E6B0E033D19A
:100220008FE71EE04DD1E0E0FAE033D180E080932B
:100230007600F9D0E0EBF9E012D3E9E6F0E010D275
:1002400084D2EDE0F0E0D8D1A1E7B0E0DC92A1E704
:10025000B0E08C91865F8C938091710080937500E3
:10026000B3D08FE717E02CD1C6D0B998A2E7B0E0A1
:100270009C9196FF04C0B19B0EC09F7B9C93B1994B
:100280000AC088E29F9399279AD19F91B19903C0A0
:1002900090649C9352D0B3CF00916800023009F073
:1002A0001BC080917200806880937200A0E6B0E06D
:1002B000E4E0FAE093D140916F00009170000417E0
:1002C00008F40AC0809172008F7780937200A0E6D4
:1002D000B0E0ECEFF9E082D100916800033009F062
:1002E0001CC080917200806880937200A0E6B0E02C
:1002F000E4E0FAE073D140916F00009170000417C0
:1003000010F009F00AC0809172008F77809372001C
:10031000A0E6B0E0ECEFF9E061D1A2E7B0E08C91AB
:1003200087FB0EF002C0C59A01C0C5988FEB1EE096
:10033000C7D0A0E6B0E0A7D020CFA8E6B0E08C916F
:100340008F5F8C9300916800033010F009F001C0BA
:1003500003C081E08093680000916800013009F0DB
:1003600005C08FE716E0ACD080E0F7D000916800C0
:10037000023009F01AC0E2E3F0E0A1E7B0E091E05A
:100380007BE7ECD28091710080936F008FE716E0DD
:1003900097D0E8E0FAE07DD08FE71EE091D081E0D1
:1003A000DCD081E0DAD081E0D8D000916800033061
:1003B00009F009C08FE71EE083D082E0CED082E052
:1003C000CCD082E0CAD00895009175004AE0DED218
:1003D000A3E7B0E00C93009173004AE0049FA4E708
:1003E000B0E00C920091750040917400041BA4E7EA
:1003F000B0E00C930895009173000A3008F003C038
:10040000E8E0FAE046D0A8E2B4E0E3E7F0E04DD25D
:1004100038D0EAE0FAE03DD0A8E2B4E0E4E7F0E06A
:1004200044D22FD00895379AEF93FF93E5E1F0E09F
:10043000BAD0FF91EF9107B1007FA6E7B0E08C91B1
:1004400090E0890F082707B9CED0A6E6B0E08D93DB
:100450009C933798E6E6F0E0D190E080FF240027F7
:1004600023D1A9E6B0E051D1E4EBF9E0F8D1E9E617
:10047000F0E0F6D0C0D1EDE0F0E0A9E6B0E05FD268
:100480000895A8E2B4E08D91882311F066D0FBCFE7
:100490000895E1D1802D11F060D0FBCF089580EC5C
:1004A00062C081E060D014D080E85DC08FE7213069
:1004B00039F08FEB223021F08FE8233009F08FECF8
:1004C000810F51C088EE93E07AD03197D9F7089523
:1004D00083E0992774C08AEF90E071D0A59AA49A1E
:1004E000A39AA29A889A899A919885E090E067D019
:1004F0009098AD98AC98AB9AAA9A909AEF93FF9384
:10050000E5E1F0E050D0FF91EF91909855D0909AAE
:10051000EF93FF93E5E1F0E046D0FF91EF919098E3
:100520004BD0909AEF93FF93E5E1F0E03CD0FF9140
:10053000EF91909841D0AA98909AEF93FF93E5E1BC
:10054000F0E031D0FF91EF91909836D088E20BD057
:100550008EE009D086E007D00895919A829505D063
:1005600004D02AD008959198F9CF859510F4AA9ACD
:1005700001C0AA98859510F4AB9A01C0AB988595F7
:1005800010F4AC9A01C0AC98859510F4AD9A01C0F6
:10059000AD98909AEF93FF93E5E1F0E004D0FF91DE
:1005A000EF91909808953197F1F70895689462F863
:1005B0000895E89462F8089581E090E000C0EF9318
:1005C000FF93EE27E82BE92B31F0EAEFF0E03197CB
:1005D000F1F70197D1F7FF91EF9108953CD10D927A
:1005E0000020E1F70895369A3699FECF369A36996B
:1005F000FECF84B195B1089533D0992711278F2D5F
:10060000880F80E8F82A802F881F08F41FEF41F038
:100610008F57082F07FD04C0003240F08FEF01C054
:100620008827982FD82EE82EF82E09C08FE1801B3E
:10063000082FF694E794D79497950A95D1F711234C
:1006400051F09095D094E094F09481E0980F882731
:10065000D81EE81EF81E0F2DFE2CED2CD92E089565
:10066000D190E190F19001910895219131914191C2
:1006700051910895102F90E8FF0C001F0927990F42
:10068000F7941078652F90E8440F551F5927990F5C
:100690004795607800380895FF0C90E89027110F77
:1006A0009795F794092F0895102FBD2CDE2CEF2C71
:1006B000F02E11234AF4B094D094E094F0949FEF7C
:1006C000B91AD90AE90AF90A0EE1FF2039F4FE2C19
:1006D000ED2CDB2CBB240850C2F76BC032F00A951E
:1006E000BB0CDD1CEE1CFF1CF9CF01D0D5CFB7FE33
:1006F000089590E8B91611F4D0FE08959FEFD91A25
:10070000E90AF90A09F403950895DD92ED92FD9244
:100710000C930895502F2D2D3E2D4F2D612F0895B0
:100720002DEC3CEC4CEC5DE366270FC099DFF2DF6B
:10073000DD24EE2490E8F92E0FE307C096DF05C014
:100740002227332740E251E46627552351F1002345
:1007500081F190DF71F11627005850580894050B6D
:1007600018F407FD03C025C007FD23C04695379543
:100770002795F694E794D79422D0FF202AF0DD0C39
:10078000EE1CFF1C015073F09D2D969548F0DD2066
:100790003AF4EE202AF491E0D90E9927E91EF91EC9
:1007A0007BCF07C09FE7092FF92A9FEFD92EE92EAB
:1007B0000895DD24EE24FF240027112708959F9239
:1007C0009924AA24BB2488E1D216E306F40628F073
:1007D000D21AE30AF40A089401C08894991CAA1C4E
:1007E000BB1CDD0CEE1CFF1C8A9571F7D92CEA2C82
:1007F000FB2C9F9008953EDFE1F25038D1F216278E
:10080000005850580894051F12F418F4CBCF08F084
:10081000D0CF0AD0FF202AF0BB0CDD1CEE1CFF1C41
:100820003BCF0F5FFBF138CF9F929924AA24BB24C2
:10083000992788E1990CAA1CBB1CDD1CEE1CFF1C2F
:1008400030F4920EA31EB41ED91EE91EF91E8A951D
:1008500089F79F900895C895319600200895FBDF91
:10086000202DF9DF302DF7DF402DF5DF502D0895D5
:10087000000F111F221F331F08950095109520951A
:1008800030950F5F1F4F2F4F3F4F089501911081FB
:100890000EC001911191219130810BC00191108105
:1008A00017FF05C03FEF2FEF04C00081112722275B
:1008B000332737FF03C0E1DF8DE28D93CF93DF93C2
:1008C000CF92DF92EF92AA24BB24CC24DD24EE2425
:1008D00040E2CAE0DD2755E093E38881890F87FD78
:1008E0009F7083FD907F891B89935A95A9F7C0DF7C
:1008F000AA1CBB1CCC1CDD1CEE1C4A9551F7E894CD
:10090000EFE0FF2782910ED0EB30E0F71EF0689405
:100910008A2D0CD088278D93EF90DF90CF90DF91B8
:10092000CF910895982F829501D0892F8F70805D87
:1009300026F0803309F4089568948D93089594E027
:1009400081918D939A95E1F70895E199FECFEEBBE1
:10095000FFBB3196089591E001C092E07B3751F4DE
:100960007FB7F894F2DF8D918DBBE29AE19A9A9568
:10097000C9F77FBF7727089591E001C092E0E5DFD6
:10098000E09A8DB38D939A95D1F70895FF93881BC4
:10099000F9E0001FFA9511F4FF910895881F841B58
:1009A00018F4840F8894F5CF0894F3CFF628DC3E32
:1009B0003333534023DBF93E5757572E4156522EBF
:1009C000344D472E434F4D200000414B5520636F5F
:1009D0006E74726F6C2056312E31000054484520E1
:1009E000454E44204F462044454D4F21000055734D
:1009F00065743D00556261743D2000004F4646001D
:0C0A0000202020004F4E200020002E007F
:00000001FF
